:10000000FFC5FFC5FFC5FFC5FFC5FFC5FFC5FFC5D0
:10001000FFC5FFC5FFC5FFC5FFC5FFC5FFC5FFC5C0
:10002000FFC5FFC5FFC5FFFFFFFFFFFFFFFFFFFF8E
:10003000FFFFFFFFFFFFFFFFFFFFFFFFFFFFFFFFD0
:10004000FFFFFFFFFFFFFFFFFFFFFFFFFFFFFFFFC0
:10005000FFFFFFFFFFFFFFFFFFFFFFFFFFFFFFFFB0
:10006000FFFFFFFFFFFFFFFFFFFFFFFFFFFFFFFFA0
:100C000012C034C033C032C031C030C02FC02EC07B
:100C10002DC02CC02BC02AC029C028C028C026C087
:100C200025C024C023C011241FBECFE5D4E0DEBF01
:100C3000CDBF8CEA90E0D4E0C0E61A92C817D9077D
:100C4000E1F710E0A0E6B0E0E4E2F7E102C00590D1
:100C50000D92A43AB107D9F710E0A4EAB0E001C0C0
:100C60001D92AC3AB107E1F7B3D15AC5C9CF1F9273
:100C70000F920FB60F921124CF92DF92EF92FF9254
:100C80002F933F934F935F936F937F938F939F9394
:100C9000AF93BF93CF93DF93EF93FF9384B195B15D
:100CA000392F20E06901EE24D7FCE094FE2C90E07F
:100CB000A0E0B0E0C82AD92AEA2AFB2A8091A40041
:100CC000882329F4C60149D281E08093A40042D24E
:100CD0008F73907081309105E9F08230910589F130
:100CE000009709F044C080918F00882349F083B5B4
:100CF0008F5F83BD83B58F3FD1F510928F0037C0D2
:100D000083B5815083BD83B5882389F581E08093C5
:100D10008F002DC080919000882349F088B58F5FA7
:100D200088BD88B58F3F19F51092900020C088B516
:100D3000815088BD88B58823D1F481E080939000EC
:100D400016C080919100882349F08AB58F5F8ABDD3
:100D50008AB58F3F61F41092910009C08AB5815025
:100D60008ABD8AB5882319F481E080939100C70178
:100D7000B60124EF31E040E050E05BD1EAE0969527
:100D8000879577956795EA95D1F72DB73EB72E50A1
:100D900030400FB6F8943EBF0FBE2DBFCDB7DEB7C3
:100DA000219620E630E0ADB7BEB712963C932E9365
:100DB000119724E630E040E050E05AD1DC01CB014D
:100DC0002A833B834C835D838E839F83A887B98767
:100DD000CA86DB86EC86FD86CBD14AB538B523B50D
:100DE000EDB7FEB736960FB6F894FEBF0FBEEDBF57
:100DF000319688E790E0ADB7BEB712969C938E937C
:100E00001197428313823483158226831782B0D1CF
:100E1000EDB7FEB738960FB6F894FEBF0FBEEDBF24
:100E2000FF91EF91DF91CF91BF91AF919F918F9102
:100E30007F916F915F914F913F912F91FF90EF9034
:100E4000DF90CF900F900FBE0F901F90189585D018
:100E500081E060E062D081E07BD086E060E05DD040
:100E600080E076D08EE060E058D080E071C0CF9313
:100E7000C82F8950823080F4CA3051F480E068D0A5
:100E800081E060E04AD080E063D082E060E045D05D
:100E900081E05ED080E805C0CD3029F481E058D0F3
:100EA00089EA60E004C080E053D08C2F61E035D047
:100EB000C093A50080E090E0CF910895C09866238C
:100EC00011F0959A01C0959895B3880F880F937C7F
:100ED000892B85BB949A82E08A95F1F700C094989B
:100EE0000895C09A94B3937C94BB882311F0959A8B
:100EF00001C09598949A82E08A95F1F700C083B377
:100F0000949894B39C6394BBC09890E08C73907059
:100F100095958795959587950895CF93DF93D82FCD
:100F2000C62F82958F70CADF8D2F8F706C2FC6DF12
:100F3000DF91CF910895CF93DF93C82FD2DFD82FC1
:100F4000D295D07F8C2FCDDF8D2BDF91CF9108955F
:100F500080E0F1DF87FDFCCF08958D9AB89A8C9AD6
:100F600084B38C6384BB8FE59AEE0197F1F700C0E0
:100F7000000083E060E0A2DF8FE090E40197F1F7EA
:100F800000C0000083E060E099DF8FE891E0019706
:100F9000F1F700C0000083E060E090DF95EC9A95E7
:100FA000F1F7000082E060E089DF80E0D1DF88E2D5
:100FB00060E0B3DF80E0CCDF88E060E0AEDF80E0BF
:100FC000C7CF85B3837C85BB9598C09894980895C6
:100FD00088E10FB6F89481BD11BC0FBEF89437DFDD
:100FE00082E990E09093AB008093AA009093A900CF
:100FF0008093A8008AE090E0CDD0BB9ABA9AB99AC3
:101000001ABC18BC81EA8FBD89E08EBD13BC89E68D
:1010100085BD17B88FEE86B9789485B78F7885BF70
:10102000F89485B7806885BF7894889585B78F7761
:10103000F6CF629FD001739FF001829FE00DF11DFA
:10104000649FE00DF11D929FF00D839FF00D749F42
:10105000F00D659FF00D9927729FB00DE11DF91FEE
:10106000639FB00DE11DF91FBD01CF01112408954B
:10107000A1E21A2EAA1BBB1BFD010DC0AA1FBB1F9C
:10108000EE1FFF1FA217B307E407F50720F0A21B0E
:10109000B30BE40BF50B661F771F881F991F1A947B
:1010A00069F760957095809590959B01AC01BD01A5
:1010B000CF0108958F929F92AF92BF92CF92DF920D
:1010C000EF92FF92CF93DF93EC0188819981AA81FF
:1010D000BB810097A105B10521F484E299EDABE550
:1010E000B7E0BC01CD012DE133EF41E050E0C6D2C5
:1010F00049015A0127EA31E440E050E09ADF6B01F0
:101100007C01C501B4012CEE34EF4FEF5FEF91DFAE
:10111000DC01CB01C80ED91EEA1EFB1EF7FE08C07B
:101120008FEF9FEFAFEFBFE7C80ED91EEA1EFB1E81
:10113000C882D982EA82FB82C6019F77DF91CF9174
:10114000FF90EF90DF90CF90BF90AF909F908F90E7
:101150000895B0CF80EA90E0ADCFA0E0B0E08093FA
:10116000A0009093A100A093A200B093A3000895C3
:10117000A0E0B0E0EDEBF8E0ACC2FE013596619185
:1011800071918091A8009091A900AF0108D020969C
:10119000E2E0BBC26091A8007091A900E5C1ADE09A
:1011A000B0E0E4EDF8E085C23C017D876C875A0130
:1011B000FC0117821682838181FFBBC12E01089436
:1011C000411C511CF3019381EC85FD8593FD8591B4
:1011D00093FF8191FD87EC87882309F4A6C18532AE
:1011E00041F493FD859193FF8191FD87EC878532D2
:1011F00021F490E0B301B8D1E5CFFF24EE2410E054
:101200001032B0F48B3269F08C3228F4803251F015
:10121000833271F40BC08D3239F0803349F41160A0
:101220002CC01260146029C0186027C0106125C04E
:1012300017FD2EC0282F20532A3098F416FF08C01F
:101240008F2D880FF82EFF0CFF0CF80EF20E15C034
:101250008E2D880FE82EEE0CEE0CE80EE20E1062DA
:101260000CC08E3221F416FD60C1106406C08C36AD
:1012700011F4106802C0883659F4EC85FD8593FDA1
:10128000859193FF8191FD87EC87882309F0B8CF82
:10129000982F9554933018F09052933038F424E0FE
:1012A00030E0A20EB31E3FE339830FC0833631F026
:1012B000833781F0833509F056C021C0F501808164
:1012C000898322E030E0A20EB31E21E0C22ED12C91
:1012D000420113C092E0292E312C2A0C3B1CF5014F
:1012E0008080918016FF03C06F2D70E002C06FEF09
:1012F0007FEFC4012ED16C0151011F7714C082E031
:10130000282E312C2A0C3B1CF5018080918016FF81
:1013100003C06F2D70E002C06FEF7FEFC4010ED1EC
:101320006C011068510113FD1AC005C080E290E005
:10133000B3011AD1EA948E2D90E0C816D906B0F305
:101340000EC0F40117FD859117FF81914F0190E0C8
:10135000B3010AD1E110EA940894C108D108C1147C
:10136000D10479F7DFC0843611F0893649F5F501EB
:1013700017FF07C080819181A281B38124E030E012
:1013800008C080819181AA2797FDA095BA2F22E0FD
:1013900030E0A20EB31E012F0F76B7FF08C0B09544
:1013A000A095909581959F4FAF4FBF4F0068BC01AE
:1013B000CD01A2012AE030E003D1D82ED4183EC0DE
:1013C000853721F41F7E2AE030E020C0197F8F3658
:1013D000A9F0803720F4883509F0A7C00BC080370A
:1013E00021F0883709F0A1C001C0106114FF09C0C5
:1013F000146007C014FF08C0166006C028E030E083
:1014000005C020E130E002C020E132E0F50117FF25
:1014100007C0608171818281938144E050E006C001
:101420006081718180E090E042E050E0A40EB51E42
:10143000A201C6D0D82ED418012F0F7706FF09C0FD
:101440000E7FDF1430F404FF06C002FD04C00F7EDF
:1014500002C01D2D01C01F2D802F90E004FF0CC085
:10146000FE01ED0DF11D2081203311F4097E09C02C
:1014700002FF06C01E5F05C086789070009709F0D5
:101480001F5F802E992403FD11C000FF0CC0FD2CAE
:101490001E1548F4FE0CF11A1E2D05C080E290E0E6
:1014A000B30162D01F5F1E15C8F304C01E1510F4EF
:1014B000E11A01C0EE2484FE0EC080E390E0B30187
:1014C00053D082FE1DC081FE03C088E590E010C0AD
:1014D00088E790E00DC0C40186789070009781F095
:1014E00081FC02C080E201C08BE207FD8DE290E04A
:1014F000B3013AD005C080E390E0B30135D0FA944F
:10150000DF14C8F3DA94F201ED0DF11D808190E053
:10151000B3012AD0DD20B1F705C080E290E0B3012D
:1015200023D0EA94EE20C9F74DCEF301868197814E
:1015300002C08FEF9FEF2D96E2E1D7C0FC0105902E
:10154000615070400110D8F7809590958E0F9F1FC5
:101550000895FC016150704001900110D8F780950A
:1015600090958E0F9F1F08950F931F93CF93DF9336
:101570008C01EB018B8181FF1BC082FF0DC02E818E
:101580003F818C819D812817390764F4E881F981B6
:101590000193F983E88306C0E885F985802F0995D2
:1015A000009731F48E819F8101969F838E8302C0C4
:1015B0000FEF1FEFC801DF91CF911F910F91089599
:1015C000FA01AA27283051F1203181F1E8946F9374
:1015D0006E7F6E5F7F4F8F4F9F4FAF4FB1E03ED01A
:1015E000B4E03CD0670F781F891F9A1FA11D680FB8
:1015F000791F8A1F911DA11D6A0F711D811D911DEB
:10160000A11D20D009F468943F912AE0269F11245F
:101610003019305D3193DEF6CF010895462F4770C3
:10162000405D4193B3E00FD0C9F7F6CF462F4F701E
:10163000405D4A3318F0495D31FD4052419302D07C
:10164000A9F7EACFB4E0A695979587957795679522
:10165000BA95C9F700976105710508959B01AC0122
:101660000A2E06945795479537952795BA95C9F749
:10167000620F731F841F951FA01D089597FB092EED
:1016800005260ED057FD04D0F3DC0AD0001C38F438
:1016900050954095309521953F4F4F4F5F4F08959E
:1016A000F6F790958095709561957F4F8F4F9F4F7E
:1016B00008952F923F924F925F926F927F928F92F6
:1016C0009F92AF92BF92CF92DF92EF92FF920F93D1
:1016D0001F93CF93DF93CDB7DEB7CA1BDB0B0FB6DB
:1016E000F894DEBF0FBECDBF09942A883988488898
:1016F0005F846E847D848C849B84AA84B984C8842E
:10170000DF80EE80FD800C811B81AA81B981CE0F24
:10171000D11D0FB6F894DEBF0FBECDBFED01089509
:10172000F894FFCF09566F6C743A20256C752E25FE
:1017300030326C752F202530346C75000D20523AF4
:101740002530327820473A2530327820423A253009
:10175000327800010101000000020000000037079C
:101760000000000001000000FFFFFFFFFFFFFFFF80
:10177000FFFFFFFFFFFFFFFFFFFFFFFFFFFFFFFF79
:10178000FFFFFFFFFFFFFFFFFFFFFFFFFFFFFFFF69
:10179000FFFFFFFFFFFFFFFFFFFFFFFFFFFFFFFF59
:1017A000FFFFFFFFFFFFFFFFFFFFFFFFFFFFFFFF49
:1017B000FFFFFFFFFFFFFFFFFFFFFFFFFFFFFFFF39
:1017C000FFFFFFFFFFFFFFFFFFFFFFFFFFFFFFFF29
:1017D000FFFFFFFFFFFFFFFFFFFFFFFFFFFFFFFF19
:1017E000FFFFFFFFFFFFFFFFFFFFFFFFFFFFFFFF09
:1017F000FFFFFFFFFFFFFFFFFFFFFFFFFFFFFF00F8
:00000001FF
